:020000040800F2
:1000000000C00020452000087D1E00087F1E00085B
:10001000811E0008831E0008851E000800000000E5
:10002000000000000000000000000000871E000823
:10003000891E0008000000008B1E00088D1E0008AD
:100040008D2000088D2000088D2000088D200008DC
:100050008D2000088D2000088D2000088D200008CC
:100060008D2000088D2000088D2000088D200008BC
:100070008D2000088D200008911E00089D1E00089C
:100080008D2000088D2000088D2000088D2000089C
:100090008D2000088D2000088D2000088D2000088C
:1000A0008D2000088D2000088D2000088D2000087C
:1000B0008D2000088D2000088D2000088D2000086C
:1000C0008D2000088D2000088D2000088D2000085C
:1000D0008D200008A91E00088D2000088D20000832
:1000E0008D2000088D2000088D2000088D2000083C
:1000F0008D2000088D2000088D2000088D2000082C
:100100008D2000088D2000088D2000088D2000081B
:100110008D2000088D200008B51E00088D200008E5
:100120008D2000088D2000088D2000088D200008FB
:1001300000000000000000000000000000000000BF
:1001400000000000000000000000000000000000AF
:10015000000000000000000000000000000000009F
:10016000000000000000000000000000000000008F
:10017000000000000000000000000000000000007F
:10018000000000000000000000000000000000006F
:10019000000000000000000000000000000000005F
:1001A000000000000000000000000000000000004F
:1001B000000000000000000000000000000000003F
:1001C000000000000000000000000000000000002F
:1001D000000000000000000000000000000000001F
:0401E0005FF8E0F1F3
:1001E40010B5054C237833B9044B13B10448AFF36D
:1001F40000800123237010BD800000200000000057
:100204004031000808B5034B1BB103490348AFF361
:10021400008008BD00000000840000204031000878
:10022400D0400B1CD1409C46203AD3401843524244
:10023400634693401843704738B50E4B054618780B
:100244004FF47A73B3FBF0F30B4A1068B0FBF3F08E
:1002540000F08EF8044658B90F2D09D802462946F5
:100264004FF0FF3000F042F8044B20461D6038BDCB
:10027400012038BD000000201800002004000020E8
:10028400074A08B51368032043F01003136000F015
:100294001BF80020FFF7D0FF01F04CFD002008BD43
:1002A40000200240034A044B11681B780B4413607E
:1002B400704700BFD004002000000020014B1868E4
:1002C400704700BFD0040020074A0002D36800F43E
:1002D400E06023F4E0631B041B0C43F0BF6343F4AE
:1002E40000330343D360704700ED00E0174B30B593
:1002F400DC68C4F30224C4F10703251D042B28BFC2
:100304000423062D4FF0010598BF002405FA03F3DA
:1003140003F1FF3388BF033C1940A14005FA04F4FC
:10032400013C2240002842EA01024FEA0212A9BF1E
:1003340000F16040064BD2B200F56140BBBF00F053
:100344000F00D2B280F800231A5430BD00ED00E053
:1003540014ED00E0002808DB0123420900F01F002F
:1003640003FA00F0014B43F82200704700E100E07B
:100374000138B0F1807F0AD2F021064B064A58605A
:1003840082F823100020072298601A607047012029
:10039400704700BF10E000E000ED00E010B5002859
:1003A40032D00168194B1424994225D8184AA3F273
:1003B40007430A44B2FBF4F2920002648468C36304
:1003C40043680A682343C46822F47F5223430469C0
:1003D40022F0300223434469234384692343C469DC
:1003E400234313430B600122002380F821208363FD
:1003F40080F82030184610BD064B0B44B3FBF4F3D1
:100404009B000364044BD9E7012010BD070402409C
:10041400F8FFFDBFF8FBFDBF00040240F0B590F803
:100424002040012C35D0012490F8215080F8204040
:10043400A5424FF000064FF0020428D180F8214075
:10044400046886632668076C26F001062660C66B7E
:10045400BD407560636043680568102BC36A0BBFB9
:10046400A260A160E160E2604BB1236843F00E0337
:1004740023602B68002043F001032B60F0BD236848
:1004840023F004032360236843F00A03F0E780F8B1
:1004940020600220F0BD000090F8213010B5022B3E
:1004A40003D004238363012010BD03681A6822F07B
:1004B4000E021A601A6822F001021A60294A934255
:1004C40024D902F56272934219D01432934218D09F
:1004D4001432934217D0143293420CBF4FF480531A
:1004E4004FF48033204A53600123002480F82130E4
:1004F400436B80F820409BB39847204610BD0123EE
:10050400F0E71023EEE74FF48073EBE717498B42D3
:1005140016D014318B4215D014318B4214D01431BF
:100524008B4214D014318B4214D014318B4214D02A
:10053400934214BF4FF480334FF080730C4AD2E7D8
:100544000123FBE71023F9E74FF48073F6E74FF438
:100554008053F3E74FF48033F0E74FF48013EDE773
:10056400184610BD8000024000040240080002400A
:100574000000024070B40425C66B026C3468036842
:1005840095402542196855D04D0753D51A689606EB
:100594005EBF1A6822F004021A60604A93421FD9AF
:1005A40002F56272934214D01432934213D014327F
:1005B400934212D0143293420CBF4FF480434FF451
:1005C4008023574A5360C36A002B00F0A58070BC97
:1005D40018470423F5E74023F3E74FF48063F0E77B
:1005E40050498B4216D014318B4215D014318B42B2
:1005F40014D014318B4214D014318B4214D01431E2
:100604008B4214D0934214BF4FF480234FF0806385
:10061400454AD7E70423FBE74023F9E74FF4806317
:10062400F6E74FF48043F3E74FF48023F0E74FF409
:100634008003EDE702259540254257D08D0755D517
:100644001A68940606D41A6822F00A021A60012273
:1006540080F82120314A93421ED902F562729342F6
:1006640013D01432934212D01432934211D0143264
:1006740093420CBF4FF400534FF40033284A5360A5
:10068400002380F82030836A9EE70223F6E72023C4
:10069400F4E74FF40073F1E722498B4216D014318A
:1006A4008B4215D014318B4214D014318B4214D0A8
:1006B40014318B4214D014318B4214D0934214BFA2
:1006C4004FF400334FF00073174AD8E70223FBE7D7
:1006D4002023F9E74FF40073F6E74FF40053F3E7F0
:1006E4004FF40033F0E74FF40013EDE7082595408D
:1006F400254211D009070FD5196821F00E011960A0
:10070400012303FA02F27260836380F8213000232C
:1007140080F82030036B57E770BC704780000240BC
:10072400000402400800024000000240114AD3685D
:1007340013F0100305D01049CB6943F00203CB61D9
:100744001023D268500706D50B4943F00403CA6945
:1007540042F00102CA61074AD169C90708D50648AF
:10076400C16941F00401C161D16921F00101D16184
:10077400D360704700200240D8040020064B18695B
:1007840010F0800007D0054A5A6002F188325A609E
:100794001869C0F3C0107047002002402301674568
:1007A400034A0020136943F080031361704700BFBC
:1007B40000200240F8B50646FFF780FD114C0746BD
:1007C4002546E368D80712D4E368990644BF20237A
:1007D400E360EB68DA0606D4EB69DB0703D4E86868
:1007E40010F0040002D0FFF7A1FF0120F8BD731C34
:1007F400E7D00EB90320F8BDFFF760FDC01B8642A9
:10080400DFD2F7E7002002402DE9F84F1F4C99464C
:10081400237E0546012B0F46904633D001234CF22C
:1008240050302376FFF7C6FF40BB012D03D0022DC5
:100834000CBF022504250026B246DFF854B032016D
:1008440040464946FFF7ECFCC4F81CA0DBF8103026
:1008540080B243F00103CBF8103027F816004CF2B5
:100864005030FFF7A7FFDBF8103023F00103CBF87B
:10087400103018B90136F3B29D42E0D80023237634
:10088400BDE8F88F0220BDE8F88F00BFD80400202F
:10089400002002400022064BDA61064B1A6942F03E
:1008A40004021A611A6942F040021A61704700BFDB
:1008B400D8040020002002400022064BDA61064BD7
:1008C4001A6942F002021A6158611A6942F0400240
:1008D4001A617047D8040020002002402DE9F0413D
:1008E400234D07462B7E8846012B3DD00124036807
:1008F4002C76022B4CF2503013D1FFF75BFF20B162
:10090400012000232B76BDE8F081FFF7C3FF4CF2F2
:100914005030FFF74FFF174A136923F004031361A4
:10092400EFE7FFF747FF0028EAD14FF0FF33C8F89D
:1009340000302046BE680F4CFA68BB6803EBC22344
:100944009E42DED23046FFF7B7FF4CF25030FFF73D
:1009540031FF236923F00203236110B1C8F800605A
:10096400CFE706F50066E7E70220BDE8F08100BFA7
:10097400D8040020002002402DE9F74F0024264629
:100984006C4F6D4BDFF8B8E1DFF8B8C10A6832FA92
:1009940006F502D103B0BDE8F08F4FF0010808FA64
:1009A40006F802EA0802904540F084804D68122D52
:1009B40000F0B18000F28780022D00F0A9807BD87E
:1009C400002D00F08C80012D00F0A0804FF00F0965
:1009D400FF2A93BF824606F18045083DD0F800B057
:1009E40092BFB500D0F804B0AD0009FA05F82BEABF
:1009F400080804FA05F588BF00F1040A48EA050569
:100A0400CAF80050D1F804A01AF0805F52D0BD6932
:100A140026F0030845F00105BD61BD6908F1804871
:100A240005F00105019508F5803806F0030B019DDA
:100A34004FEA8B0BD8F8085009FA0BF925EA090993
:100A44003E4DA8426CD005F58065A8426AD005F5F4
:100A54008065A84268D005F58065A84266D005F592
:100A64008065A84264D070450CBF0525062505FAAB
:100A74000BF545EA0905C8F808501D681AF4803FCB
:100A840014BF154395431D605D681AF4003F14BFFD
:100A9400154395435D609D681AF4801F14BF154388
:100AA40095439D60DD681AF4001F14BF2A4325EAAC
:100AB4000202DA60013669E7032D25D0112D85D1B4
:100AC400CC68043482E7654509D012D8DFF8789001
:100AD4004D4504D009F580394D457FF477AF8C68D6
:100AE400E4B1012C0CBFC0F81080C0F814800824B5
:100AF4006CE7DFF858904D45F1D009F580394D4544
:100B0400EDD0A9F58019E7E700245FE7CC685DE73D
:100B1400CC6808345AE7CC680C3457E7042455E70A
:100B24000025A4E70125A2E70225A0E703259EE707
:100B340004259CE700100240000401400008014025
:100B4400001C0140000021100000111000003110B1
:100B54000AB1016170470904FBE7C3680B4214BF83
:100B640041610161704700002DE9F341054608B970
:100B740001203CE00368DB0710D42B689F075DD499
:100B84002B68190700F194802B685A0700F1BE8086
:100B9400E869002840F02C81002028E08F4C63682D
:100BA40003F00C03042B07D0636803F00C03082B39
:100BB40009D16368DE0306D523689C03DDD56B6821
:100BC400002BDAD1D4E76B68B3F5803F12D12368E8
:100BD40043F480332360FFF771FB064623689803D0
:100BE400CBD4FFF76BFB801B6428F7D9032002B03A
:100BF400BDE8F0819BB9236823F480332360236824
:100C040023F480232360FFF759FB064623689903E6
:100C1400B3D5FFF753FB801B6428F7D9E6E7B3F598
:100C2400A02F236803D143F480232360CFE723F468
:100C340080332360236823F48023CBE7674C636805
:100C440013F00C0F07D0636803F00C03082B10D1CA
:100C54006368DA030DD423689B0702D52B69012B43
:100C640086D123686A6923F0F80343EAC203236048
:100C740086E72A695A4B6AB101221A60FFF71EFB04
:100C8400064623689F07ECD4FFF718FB801B022855
:100C9400F7D9ABE71A60FFF711FB064623689807FC
:100CA4007FF56EAFFFF70AFB801B0228F6D99DE79C
:100CB400AA694A4C4B4BDAB101221A60FFF7FEFADB
:100CC4000646636A9B070DD54FF4FA52464B1B68E0
:100CD400B3FBF2F3019300BF019B5A1E0192002B58
:100CE400F9D151E7FFF7EAFA801B0228E9D97DE739
:100CF4001A60FFF7E3FA0646636A9F077FF544AF7D
:100D0400FFF7DCFA801B0228F6D96FE7334CE3695E
:100D1400D80024D40127E36943F08053E361E369F5
:100D240003F080530093009B304E3368D90518D5E7
:100D3400EB68012B26D1236A43F001032362FFF7FA
:100D4400BDFA41F288368046236A9B073FD5002FBF
:100D54003FF41EAFE36923F08053E36118E70027F3
:100D6400E2E7336843F480733360FFF7A7FA804601
:100D74003368DA05DCD4FFF7A1FAA0EB0800642895
:100D8400F6D933E7ABB9236A41F2883823F001037B
:100D94002362236A23F004032362FFF78FFA0646D3
:100DA400236A9807D3D5FFF789FA801B4045F7D902
:100DB4001CE7052B236A03D143F004032362BAE73B
:100DC40023F001032362236A23F00403B6E7FFF749
:100DD40075FAA0EB0800B042B6D907E7001002404C
:100DE400000042428004424218000020007000408B
:100DF4002A4B5A681C4602F00C02082A3DD00023F4
:100E0400274E022833602BD1FFF758FA0746236890
:100E140099011FD42B6AB3F5803F05D16268A96894
:100E240022F400320A436260696A62680B4322F466
:100E340074121343636001233360FFF73FFA0546DE
:100E440023689A013FF5A8AEFFF738FA401B022841
:100E5400F6D9CBE6FFF732FAC01B0228D7D9C5E68C
:100E6400FFF72CFA054623689B017FF595AEFFF743
:100E740025FA401B0228F6D9B8E601283FF4B7AE9C
:100E840058682B6A00F480329A427FF471AE6B6A20
:100E940000F47010C01A18BF0120A8E60010024028
:100EA4006000424230B5194B87B002AC03F1100523
:100EB400224618685968083303C2AB421446F7D176
:100EC40001238DF80430022311498DF805304B6855
:100ED40003F00C02082A17D1C3F3834206A8024484
:100EE400DB0312F8102C0CD54B680A48C3F34043BB
:100EF400504306AA134413F8143CB0FBF3F007B0B4
:100F040030BD05485043FAE70248F8E75831000875
:100F14000010024000127A0000093D002DE9F04162
:100F24000D46044610B90120BDE8F081454A136816
:100F340003F007038B4229D321688E0731D4CA07F3
:100F440044D4404A136803F007039D4267D32268E0
:100F54003D4D12F0040F6ED1130706D56B6822695C
:100F640023F4605343EAC2036B60FFF79BFF6B6893
:100F7400364AC3F30313D35CD840354B1860354B62
:100F84001868FFF759F90020BDE8F081136823F0D1
:100F940007030B431360136803F007039942C2D19C
:100FA400CAE7294B11F0040F1EBF5A6842F4E062ED
:100FB4005A60080742BF5A6842F460525A605A683D
:100FC400A06822F0F00202435A60B8E762681E4E3D
:100FD400012A33681BD113F4003FA4D0736841F293
:100FE400883823F0030313437360FFF767F9074658
:100FF4007368626803F00C03B3EB820FA1D0FFF7B0
:101004005DF9C01B4045F3D90320BDE8F081022AF5
:1010140002D113F0007FE0E713F0020FDDE713685D
:1010240023F007032B431360136803F007039D4267
:101034007FF479AF8BE76B68E16823F4E0630B43DB
:101044006B6089E70020024000100240C3310008B1
:101054001800002004000020044B054A5B68C3F319
:101064000223D35C034A1068D84070470010024042
:10107400D331000818000020044B054A5B68C3F311
:10108400C223D35C034A1068D84070470010024062
:10109400D33100081800002003680020DA6842F009
:1010A4000102DA609A6802F00702062A1EBF1A6873
:1010B40042F001021A6070477047704770477047EA
:1010C400036810B51A69044691070ED5DA689207C9
:1010D4000BD56FF002021A6101229B6902779B070C
:1010E40077D0FFF7EAFF0023237723681A695007B4
:1010F40010D5DA6851070DD56FF004021A61022287
:101104009B69227713F4407F204668D0FFF7D5FF10
:101114000023237723681A6912070FD5DA681007AA
:101124000CD56FF008021A610422DB692277990753
:1011340020465AD0FFF7C1FF0023237723681A699A
:10114400D20610D5DA68D0060DD56FF010021A61F8
:101154000822DB69227713F4407F20464BD0FFF747
:10116400ACFF0023237723681A69D10708D5DA680E
:10117400D20705D56FF0010220461A6100F0BAFCCF
:1011840023681A69100608D5DA68110605D56FF0C8
:10119400800220461A6100F0BAF823681A695206E0
:1011A40008D5DA68500605D56FF0400220461A616A
:1011B400FFF785FF23681A69910622D5DA6892063B
:1011C4001FD56FF020022046BDE810401A6100F0E0
:1011D4009DB8FFF771FF2046FFF770FF83E7FFF725
:1011E4006BFF2046FFF76AFF92E7FFF765FF204693
:1011F400FFF764FFA0E7FFF75FFF2046FFF75EFFFE
:10120400AFE710BD244A0368904212D002F5006291
:1012140090420ED0B0F1804F0BD0A2F5983290429C
:1012240007D002F58062904203D002F580629042BA
:101234001DD14A6823F070031343174A904212D019
:1012440002F5006290420ED0B0F1804F0BD0A2F5AF
:101254009832904207D002F58062904203D002F5A2
:101264008062904203D1CA6823F4407313434A69ED
:1012740023F08003134303608B68C3620B688362AB
:10128400054B984203D003F50063984201D10B69E2
:101294000363012343617047002C014010B50446E9
:1012A400A0B190F83D3003F0FF021BB980F83C2058
:1012B40000F062FD0223206884F83D30211DFFF711
:1012C400A1FF0123002084F83D3010BD012010BD92
:1012D40090F83C3030B5012B4FF0020314D0046871
:1012E40080F83D306268A3680D68496822F0700296
:1012F40023F080030B432A436260A360012380F838
:101304003D30002380F83C30184630BD70477047AC
:101314000368DA6822F49072DA605A6922F00102F2
:101324005A61202380F83A307047000038B50546EA
:101334000368C1681A69192422F440520A431A61E5
:1013440082680069D9680243686921F4B05121F0C8
:101354000C0102430A43DA605A69A96922F4407213
:101364000A435A610D4A934214D1FFF785FE604344
:101374006C686422A400B0FBF4F0B0FBF2F402FB4E
:1013840014031B013233B3FBF2F3296803EB041398
:101394008B6038BDFFF760FEE9E700BF003801400D
:1013A400F8B504460E4617461D4621680B6836EA12
:1013B400030301D10020F8BD6B1CF7D095B9236855
:1013C4000320DA6822F4D072DA605A6922F001024A
:1013D4005A61202384F8393084F83A30002384F8A1
:1013E4003830F8BDFEF76AFFC01B8542DDD2E6E760
:1013F40010B5044640B390F8393003F0FF021BB92E
:1014040080F8382000F0CCFC2423226884F839309A
:10141400D368204623F40053D360FFF787FF236883
:1014240000201A6922F490421A615A6922F02A02B1
:101434005A61DA6842F40052DA602023E06384F8E7
:10144400393084F83A3010BD012010BD2DE9F04147
:101454001F4690F839300446202B0D4690464ED155
:10146400002949D0002A47D090F83830012B46D0C3
:10147400012380F838300023C363212380F83930F6
:10148400FEF71CFF0646A4F82480A4F82680E38C0B
:101494009BB26BB93B46324640212046FFF780FFA2
:1014A400A8B9202384F8380084F83930BDE8F081E5
:1014B400E38C3246013B9BB2E384A3688021B3F5FD
:1014C400805F20463B460ED1FFF76AFF10B1032030
:1014D400BDE8F0812B882268C3F3080353602369B5
:1014E40043B90235D3E7FFF75BFF0028EFD1236848
:1014F4002A785A600135CAE70120BDE8F08102204C
:10150400BDE8F08138B50446134694F83920202A02
:101514002AD139B333B394F83820012A24D00122D4
:10152400002584F838202122E384206BE56384F8C5
:1015340039200E4AA384216282620D4A4563C26245
:101544000C4A026322680432FEF768FF6FF040021F
:10155400236828461A605A6984F8385042F0800299
:101564005A6138BD012038BD022038BD0F1600086D
:101574003D16000809170008134690F83A2073B581
:10158400202A054638D1002934D0002B32D090F8D7
:101594003820012A30D00122002480F83820222269
:1015A40081628385C46380F83A20406B134A2E68B5
:1015B4008262134A4463C262124A02630A46311DBC
:1015C400FEF72CFF20462B6801941A6801925A6892
:1015D40085F838400192019ADA6842F48072DA6040
:1015E4005A6942F001025A615A6942F040025A6152
:1015F40002B070BD0120FBE70220F9E7471600089E
:10160400FD16000809170008704708B50368426A08
:101614001B6813F020030AD1D38413685A6922F09B
:1016240080025A61DA6842F04002DA6008BD10466E
:10163400FFF7EAFF08BD704708B5406AFFF7FBFFF4
:1016440008BD08B50368426A1B6813F0200310D173
:10165400D3851368D96821F48071D960596921F060
:1016640001015961596921F040015961202382F82F
:101674003A30104600F0B6FC08BD90F83A3010B588
:10168400222B36D183680169B3F5805F0268836ACF
:1016940023D15268E9B9C2F3080223F8022B83620A
:1016A400C48D013CA4B2C4858CB90368DA6822F005
:1016B4002002DA60DA6822F48072DA605A6922F071
:1016C40001025A61202380F83A3000F08BFC00209C
:1016D40010BDD2B223F8012BE1E721B9591C52689D
:1016E40081621A70DCE75268591C816202F07F0241
:1016F400F7E7022010BD704708B5406AFFF7FBFF0B
:1017040008BD7047416A08B50B685A6991F83900F9
:1017140021280AD1120608D50022CA84DA6822F0E8
:10172400C002DA60202281F839205B6991F83A20FE
:10173400222A06D15B0604D500230846CB85FFF791
:10174400E7FDCB6B084643F01003CB63FFF7D9FFEB
:1017540008BD0000036870B51A6804461607D96806
:101764005D6907D196065AD58D0658D5BDE87040F7
:10177400FFF783BF15F0010502D111F4907F4ED01D
:10178400D30705D5CE0542BFE36B43F00103E36302
:10179400500704D51DB1E36B43F00203E3639307E1
:1017A40004D51DB1E36B43F00403E363160704D5CA
:1017B4001DB1E36B43F00803E363E36B002B66D0D6
:1017C400950604D5880602D52046FFF756FF236800
:1017D40020465D69E26B110702D415F040051AD06A
:1017E400FFF796FD23685A69520610D55A69606B53
:1017F40022F040025A6150B1254B4363FEF74CFE80
:10180400002844D0606BBDE87040436B1847204605
:10181400FFF777FF70BDFFF774FFE56370BD160631
:1018240027D50D0625D594F83920212A2FD1A26871
:10183400B2F5805F226A17D11188C1F3080159609B
:10184400216979B902322262E28C013A92B2E284CD
:10185400EAB9DA6822F08002DA60DA6842F040021B
:10186400DA6070BD0132EEE7511C216212785A60D1
:10187400EAE750060BD54A0609D5DA68204622F075
:101884004002DA60202384F83930FFF7BDFE70BDD2
:101894009918000808B50023406AC385C384FFF77C
:1018A40030FF08BD10B5064CA178601C00F05CF850
:1018B400A178207103312046BDE8104000F0B8BB88
:1018C4000E00002070B58178044643185A78013020
:1018D40000F065F8C0B201280ED000231E4EA27895
:1018E4005D1C0232DBB29A422EDA1C4800F074FC12
:1018F40022221B4B5A700FE01122194D6A70627834
:10190400DD2A01D0EE2A07D1204600F0B7F8C0B294
:10191400012801D122236B70114DA978681C00F0B5
:1019240023F828716378EE2B06D00A2B04D0A9780B
:101934002846033100F07CFB6378EE2B0AD1BDE826
:101944007040084800F048BCE15C304600F0D0FB31
:101954002B46C4E770BD00BF683100086E31000833
:10196400080000207F31000810B5FF230446221A26
:10197400D2B2914201D8184610BD14F8012B53403D
:10198400082213F0800F02F1FF324FEA430318BF1D
:1019940083F0310312F0FF02DBB2F2D1E7E730B596
:1019A400FF2305462C1AE4B2A14203D89B1A5842DD
:1019B400584130BD15F8014B6340082413F0800FE3
:1019C40004F1FF344FEA430318BF83F0310314F0EA
:1019D400FF04DBB2F2D1E5E70C4A10B5D3690C4839
:1019E40023F01003D36100F0F7FB0A4B0A4A1B688B
:1019F4000A4C0B481360236000F0EEFB094B1B6894
:101A040083F308882368BDE810401847001002409B
:101A1400AB31000804400008F8040020FC04002056
:101A2400BD310008004000082DE9F04100240746BC
:101A34002646104DDFF84080BB78023B9C4202DB17
:101A44003046BDE8F0813B19DA781B79296802EB4E
:101A5400032292B200230120FEF7D6FE18B14046BD
:101A640000F0BAFB01262B68023402332B60E4B287
:101A7400E2E700BF1400002090310008002373B592
:101A8400164D174C2B60174B0646AB601F23EB60BB
:101A9400E36923F01003E361FEF770FE124B1A783A
:101AA4004AB90122114928461A70FEF717FF10B1EE
:101AB4000F4800F091FB3046FFF7B6FF0546FEF7EE
:101AC4006FFE2846E36943F01003E361E36903F022
:101AD40010030193019B02B070BD00BF9C00002065
:101AE4000010024000400008B0000020AC000020BC
:101AF4009C3100080268084B9A420BD1074A1368CC
:101B040001331360064A136801331360054A1368EE
:101B140001331360704700BF00100040BC00002078
:101B2400B8000020B400002010B514460A2302486F
:101B3400FFF78CFC204610BD8805002010B590B03E
:101B44002822002106A800F0CBFA1422002101A8C3
:101B540000F0C6FA01230A93102302240B934FF4D6
:101B6400601306A806940D940F93FEF7FDFF00B1D1
:101B7400FEE70F2301934FF4806303900590214601
:101B840001A802940493FFF7C9F900B1FEE710B06D
:101B940010BD000080B588B0FEF772FBFFF7CEFFE2
:101BA4001022584C00210DEB020000F099FAA369B1
:101BB400002243F01003A361A3694FF4004103F032
:101BC40010030293029BA3694F4843F00403A361EB
:101BD400A369002603F004030393039BFEF7B8FFF5
:101BE4004FF400430493012305930223464804A9B8
:101BF40007930696FEF7C0FE6369444D43F0010364
:101C040063616369424803F001030193019B41F658
:101C1400FF0385E809000923284604960596AE606B
:101C2400EB60AE61FFF73AFB00B1FEE7049005906C
:101C340004A92846FFF74CFB00B1FEE74FF4E1325C
:101C4400344B3549986083E806000C22D86018614B
:101C54009861D86118465A61FFF7CAFB044600B17F
:101C6400FEE7024601463620FEF740FB3620FEF72B
:101C740071FB224621462520FEF738FB2520FEF77E
:101C840069FB224621460F20FEF730FB0F20FEF7AA
:101C940061FB224621460E20FEF728FB0E20FEF7AC
:101CA40059FB2846FFF7F8F91C4B21461B68164ED2
:101CB400986800F099FAFFF7F5FD194800F058F913
:101CC400184D194C2368642B06D94FF40041304653
:101CD400FEF743FF00232360114C0E4FA368002B33
:101CE40002DD2B681E2B03D8104F40F6B83405E0F4
:101CF400384600F04BF9F1E7FFF76EFE3B68A3426C
:101D0400FAD8DEE70010024000100140C8050020A8
:101D14000010004088050020003801401C0000200D
:101D240008060020BC000020B8000020B4000020F9
:101D3400FEE700000E4B82B09A6942F001029A61FC
:101D44009A6902F001020092009ADA6942F0805224
:101D5400DA61DB69074A03F080530193019B5368FE
:101D640023F0E06343F08063536002B0704700BF28
:101D740000100240000001400268084B82B09A4201
:101D84000AD103F50033DA6942F01002DA61DB6943
:101D940003F010030193019B02B070470010004050
:101DA40070B5064686B01022002102A800F098F90A
:101DB40032682B4B9A4251D103F558439A6902A9D0
:101DC40042F480429A619A69264802F48042009261
:101DD400009A9A69002542F004029A619B69224C98
:101DE40003F004030193019B4FF400730293022355
:101DF400039303230593FEF7BFFD4FF48063194853
:101E040002A9029303950495FEF7B6FD174B2046ED
:101E140084E828008023A560E36025616561A561ED
:101E2400E561FEF7BBFA08B1FFF782FF4FF0100C33
:101E34000F4B746366620F4C802284E80810002301
:101E44002046A360E26023616361A361E361FEF75E
:101E5400A5FA08B1FFF76CFF3463666206B070BD83
:101E640000380140000801404405002058000240A9
:101E740044000240000500207047FEE7FEE7FEE74D
:101E8400FEE7704770477047FEF70CBA0148FEF74B
:101E940071BB00BF000500200148FEF76BBB00BF0B
:101EA400440500200148FFF755BC00BF8805002009
:101EB4000148FFF705B900BFC805002070B50E46FC
:101EC40015460C46A31B9D4201DC284670BDAFF3AA
:101ED400008004F8010BF5E708B50A4B02461968BF
:101EE40009B9094919606946186802448A4206D941
:101EF40000F0CCF80C2303604FF0FF3008BD1A60EB
:101F040008BD00BFC0000020180A00204FF0FF30B9
:101F140070474FF4005300204B6070470120704716
:101F2400002070470F4B1A6842F001021A6059688A
:101F34000D4A0A405A601A6822F0847222F48032F0
:101F44001A601A6822F480221A605A6822F4FE0287
:101F54005A604FF41F029A604FF00062034B9A607C
:101F6400704700BF001002400000FFF800ED00E0E1
:101F74000023012243600360836002490248FFF7A3
:101F8400FBBA00BF1406002088050020114A38B5AA
:101F94001468631C1360104B596803F10C000D5C4A
:101FA4000131B1F5806FA8BF00210C485960055577
:101FB4009C680546013C9C605CB908481460FFF7C6
:101FC40081FC23462B550134B4F5806FFAD1044AC1
:101FD400136038BDC400002008060020C80000209B
:101FE400B4000020002310B50D4A0E4C1360226883
:101FF4000132B2F5806FB8BF13462360A368013382
:10200400B3F5806FA36001DBFFF7C0FF23680649C7
:102014000122BDE8104019440448FFF7ADBA00BFDF
:10202400BC000020080600201406002088050020BB
:102034000A4601460148FFF765BA00BF880500203B
:10204400002103E00B4B5B58435004310A480B4B0F
:1020540042189A42F6D30A4A02E0002342F8043BAB
:10206400084B9A42F9D3FFF75DFF00F015F8FFF72C
:1020740091FD70477C3200080000002080000020A1
:1020840080000020180A0020FEE70000014B1868B9
:10209400704700BF1C00002070B500250C4E0D4C8D
:1020A400A41BA410A54209D101F048F800250A4E4A
:1020B4000A4CA41BA410A54205D170BD56F82530C6
:1020C40098470135EEE756F8253098470135F2E791
:1020D4007432000874320008743200087832000840
:1020E40003460244934200D1704703F8011BF9E709
:1020F4000FB40A4B13B51C6824B1A36913B9204665
:1021040000F0DAFA05AB049AA1682046019300F0C6
:102114009BFC02B0BDE8104004B070471C000020D6
:1021240070B50E46054618B183690BB900F0C4FAC0
:10213400AB69AC6813B9284600F0BEFA234B9C4245
:1021440017D16C68A3891B071DD52369DBB1013E38
:10215400A36816F8011F013BA360E9B9002B2EDA2E
:1021640022460A21284600F0F5F8013011D00A2051
:1021740070BD174B9C4201D1AC68E3E7154B9C4200
:1021840008BFEC68DEE72146284600F035F9002850
:10219400DDD04FF0FF3070BD002B04DAA26993420A
:1021A40006DB0A2904D023685A1C22601970CFE781
:1021B4002246284600F0CEF80130C9D1E9E70A20CA
:1021C40023685A1C2260187070BD00BF00320008DA
:1021D40020320008E0310008024B01461868FFF77E
:1021E4009FBF00BF1C00002000294FF480630CBF78
:1021F4000222002200F000B82DE9F7431D46514B9E
:1022040004461E680F46904626B1B36913B930469A
:1022140000F052FA4C4B9C4252D17468B8F1020F50
:1022240006D0B8F1010F00F28980002DC0F286803B
:102234002146304600F0D6F9616B41B104F1440304
:10224400994202D0304600F02DFB00236363002343
:10225400A3616360A3891B0603D52169304600F09E
:1022640021FBA389B8F1020F23F44A6323F003038B
:10227400A3815DD001AB6A462146304600F0A6FA40
:10228400A3891843A0812DBB009D284600F002FBC2
:10229400074600284ED1DDF80090A9453CD14FF007
:1022A400FF30A38943F00203A3810023A36004F158
:1022B4004703236023610123636103B0BDE8F08316
:1022C400224B9C4201D1B468A8E7214B9C4208BF31
:1022D400F468A3E7002FD8D0B36913B9304600F0EF
:1022E400EBF9B8F1010F08BFA389276004BF43F0DD
:1022F4000103A381A389276113F0080065611BD042
:1023040013F001004FF000031FBF6D42A360A561ED
:10231400184608BFA560D0E7484600F0BBFA074658
:102324000028BCD0A3894D4643F08003A381D3E7A2
:102334000020B6E7A946F5E7A060BEE74FF0FF30FE
:10234400BBE700BF1C000020003200082032000858
:10235400E0310008F8B50E461446054618B1836905
:102364000BB900F0A9F9214B9C422AD16C68A369EE
:10237400A360A3891A072ED5236963B32369206850
:10238400F6B2C01A63693746984204DB21462846F0
:1023940000F028F928BBA3680130013BA36023683F
:1023A4005A1C22601E706369984204D0A389DB071B
:1023B40019D50A2E17D12146284600F013F990B1F9
:1023C4000FE00B4B9C4201D1AC68D0E7094B9C4217
:1023D40008BFEC68CBE72146284600F00DF800283A
:1023E400CCD04FF0FF373846F8BD00BF00320008AC
:1023F40020320008E0310008324B70B51D680646F3
:102404000C4625B1AB6913B9284600F055F92E4B9B
:102414009C420FD16C68B4F90C309AB215072CD4D5
:10242400D00611D40922326043F04003A3814FF057
:10243400FF3070BD254B9C4201D1AC68EBE7244BC7
:102444009C4208BFEC68E6E7510712D5616B41B1C5
:1024540004F14403994202D0304600F023FA0023E9
:102464006363A38923F02403A381002363602369A6
:102474002360A38943F00803A38123694BB9A3898B
:1024840003F42073B3F5007F03D02146304600F0F7
:10249400C1F9A28912F001030CD00023A36063697F
:1024A4005B42A361236953B9B4F90C3013F0800083
:1024B400BAD170BD920758BF6369A360F2E70020E8
:1024C400F7E700BF1C00002000320008203200089B
:1024D400E03100088A892DE9F041054610070C46D1
:1024E4005AD44B68002B05DC0B6C002B02DC00205B
:1024F400BDE8F081E66A002EF9D0002312F4805280
:102504002F682B6033D0606DA3895A0705D56368A3
:10251400C01A636B0BB1236CC01A00230246E66A2F
:10252400216A2846B047431CA38906D129681D297E
:102534004BD82B4ACA40D60747D50022626022698D
:10254400D904226004D5421C01D12B6803B960650B
:10255400616B2F600029CAD004F14403994202D070
:10256400284600F09FF900206063BDE8F081216AED
:1025740001232846B047411CC6D12B68002BC3D089
:102584001D2B01D0162B01D12F60B0E7A38943F096
:102594004003A381BDE8F0810F69002FA7D0930702
:1025A40018BF00230E6808BF4B69A6EB07080F602D
:1025B4008B60B8F1000F9ADD43463A46216A2846FB
:1025C400A66AB047002807DCA38943F04003A3812F
:1025D4004FF0FF30BDE8F0810744A8EB0008E8E7BE
:1025E4000100402038B50B6905460C46DBB118B133
:1025F40083690BB900F060F80C4B9C4209D16C68FC
:10260400B4F90C307BB121462846BDE83840FFF7C9
:1026140061BF074B9C4201D1AC68F1E7054B9C427A
:1026240008BFEC68ECE7002038BD00BF00320008AA
:1026340020320008E0310008014900F0A9B800BFC9
:10264400E9250008002310B5044603604360836055
:1026540081814366C2810361436183611946082213
:102664005C30FFF73DFD054B24626362044BA362BB
:10267400044BE362044B236310BD00BFC92F000861
:10268400EB2F0008233000084730000870B5682598
:102694004A1E55430E4605F1740100F04FF90446F5
:1026A40040B1002180E842000C30A06005F16802CE
:1026B400FFF716FD204670BD836910B5044633BB91
:1026C4008364C3640365124B124A1B688262984296
:1026D40004BF0123836100F01FF86060204600F00E
:1026E4001BF8A060204600F017F80022E0600421E7
:1026F4006068FFF7A7FF01220921A068FFF7A2FF86
:1027040002221221E068FFF79DFF0123A36110BD9F
:10271400DC3100083D260008F8B51C4B07461E684E
:10272400B36913B93046FFF7C7FF4836B468736816
:10273400013B03D5336833B13668F7E7B4F90C507D
:102744006DB16834F4E704213846FFF79FFF306029
:102754000028F1D10C2304463B602046F8BD4FF617
:10276400FF73E38101236566A3812560A56065602D
:1027740025616561A5610822294604F15C00FFF723
:10278400AFFC6563A563A564E564E6E7DC31000896
:102794002DE9F84380468946002600F1480414B91F
:1027A4003046BDE8F883A5686768013F01D5246811
:1027B400F5E7AB89012B07D9B5F90E30013303D006
:1027C40029464046C84706436835EEE770B50E46CD
:1027D400B1F90E1090B0002914461D4607DA002303
:1027E4002B60B3891A0610D44FF480630EE001AA5B
:1027F40000F04EFC0028F2DB029A02F47042A2F5CB
:1028040000535A425A412A60EEE7402300202360D5
:1028140010B070BD8B8973B59D0706460C4607D56D
:1028240004F14703236023610123636102B070BD97
:1028340001AB6A46FFF7CAFF00990546304600F02F
:102844007DF848B9B4F90C309A05EFD423F00303AA
:1028540043F00203A381E3E70D4BB362A389206035
:1028640043F08003A381009B20616361019B5BB102
:10287400B4F90E10304600F01DFC28B1A38923F0F2
:10288400030343F00103A381A3891D43A581CDE77D
:102894003D260008024B0146186800F04FB800BFFF
:1028A4001C00002038B50546002943D051F8043CEB
:1028B4000C1F002BB8BFE41800F02CFC1E4A136850
:1028C400104633B9636014602846BDE8384000F010
:1028D40022BCA3420BD921686218934201BF1A6833
:1028E4005B685218226063600460EDE713465A681F
:1028F4000AB1A242FAD919685818A0420BD120682B
:102904000144581882421960DED1106852680144AB
:1029140019605A60D8E702D90C232B60D4E72068E9
:1029240021188A4201BF1168526809182160626047
:102934005C60C9E738BD00BFC804002070B5CD1C79
:1029440025F0030508350C2D38BF0C25002D06464F
:1029540001DBA94203D90C233360002070BD00F0D1
:10296400D9FB234A1468214691B9224C23681BB928
:10297400304600F017FB20602946304600F012FB79
:10298400431C26D10C233046336000F0C4FBE4E73B
:102994000B685B1B1AD40B2B0FD90B60CC18CD50D2
:1029A400304600F0B8FB04F10B00231D20F00700B3
:1029B400C31A1BD05A42E25070BD8C420BBF6368ED
:1029C4004B681360636018BF0C46E9E70C4649681E
:1029D400CAE7C41C24F00304A04205D0211A3046DF
:1029E40000F0E0FA0130CDD02560D9E770BD00BF1A
:1029F400C8040020CC040020936810B4013B002BD1
:102A0400936008DA9469A34202DBCBB20A2B02D1A9
:102A140010BCFFF79FBC1368581C10601970C8B233
:102A240010BC7047F8B506460F461446D518AC429C
:102A340001D1002007E03A4614F8011B3046FFF7A5
:102A4400DBFF431CF3D1F8BD2DE9F04F9DB00C46DC
:102A540017460393064618B183690BB9FFF72CFE9A
:102A64007C4B9C4257D17468A38918075DD52369B0
:102A7400002B5AD00023099320238DF829303023CA
:102A84004FF0010B8DF82A30B846454615F8013B46
:102A9400002B55D1B8EB070A0BD053463A462146D2
:102AA4003046FFF7BFFF013000F0C480099B534458
:102AB400099398F80030002B00F0BC8000234FF0FD
:102AC400FF3204930793059206938DF853301A93BB
:102AD40005222978604800F00FFB05F10108049BEA
:102AE400002831D1D90644BF20228DF853201A077B
:102AF40044BF2B228DF853202A782A2A2CD0002177
:102B04000A20079AA84698F800300135303B092B73
:102B14006DD971B326E0514B9C4201D1B468A3E74F
:102B24004F4B9C4208BFF4689EE721463046FFF7AE
:102B340063FC00289ED04FF0FF301DB0BDE8F08F3D
:102B4400252BA7D0A846A0E7434A4546801A0BFA8E
:102B540000F018430490BBE7039A111D1268039117
:102B6400002A01DB079204E0524243F00203079279
:102B7400049398F800302E2B10D198F8013008F106
:102B840001012A2B37D1039B08F102081A1D1B6887
:102B94000392002BB8BF4FF0FF330593314D03224E
:102BA40098F80010284600F0A7FA40B14023401BD3
:102BB40003FA00F0049B08F101080343049398F816
:102BC40000100622284808F101078DF8281000F0AB
:102BD40093FA002834D0254B03BB039B073323F01F
:102BE400070308330393099B4B4409934CE700FB09
:102BF4000232012186E700230A25184605938846F8
:102C040098F800200131303A092A03D9002BC5D0A5
:102C14000590C3E705FB00200123F0E703AB009315
:102C24002246134B04A93046AFF30080B0F1FF3FB6
:102C34008146D8D1A3895B063FF57DAF09987CE72F
:102C440003AB009322460A4B04A9304600F08AF8ED
:102C5400ECE700BF003200084032000820320008D0
:102C6400E0310008463200084A3200080000000043
:102C7400292A00082DE9F04791461F468A680B6906
:102C840006469342B8BF1346C9F8003091F8432072
:102C94000C46DDF8208012B10133C9F800302368F6
:102CA400990642BFD9F800300233C9F800302568CC
:102CB40015F0060507D104F1190AE368D9F80020D4
:102CC4009B1A9D422ADB94F843302268003318BFD4
:102CD400012392062FD404F1430239463046C047FB
:102CE400013022D02368E56803F00603042B18BFE3
:102CF4000025D9F800204FF0000908BFAD1AA368D9
:102D0400226908BF25EAE5759342C4BF9B1AED18F2
:102D14001A344D451BD10020BDE8F08701235246EB
:102D240039463046C047013003D14FF0FF30BDE88B
:102D3400F0870135C1E73020E11881F843005A1CBF
:102D440094F845102244023382F84310C3E7012368
:102D5400224639463046C0470130E6D009F1010920
:102D6400D7E700002DE9F04317460A7E85B06E2AA6
:102D7400984606460C460C9B01F1430E00F0BC80BD
:102D84001AD8632A2ED00AD8002A00F0C880582AFC
:102D940000F08A8004F1420584F842202AE0642A83
:102DA40001D0692AF6D121681A6811F0800F23D066
:102DB400111D1960136827E0732A00F0B48008D845
:102DC4006F2A2AD0702AE5D10A6842F020020A60EC
:102DD40003E0752A21D0782ADCD178226F4984F85F
:102DE400452064E01A6801F14205111D1960136859
:102DF40084F842300123A3E011F0400F02F10401F2
:102E04001960D7D0B2F90030002B03DA2D225B42CF
:102E140084F8432062490A2217E02068196810F0F8
:102E2400800F03D0081D18600B6806E010F0400FF7
:102E340001F104001860F7D00B886F2A14BF0A222E
:102E440008225749002084F843006568002DA560D6
:102E5400C0F29C80206820F004002060002B3FD149
:102E6400002D40F095807546082A0BD12368DA07B7
:102E740008D5236962689A42DEBF302305F8013C15
:102E840005F1FF35AEEB05032361CDF800803B4629
:102E940003AA21463046FFF7EDFE013055D14FF02D
:102EA400FF3005B0BDE8F08381F845203C49226835
:102EB400186812F0800F00F104051D6001D003684A
:102EC40002E05506FBD50388D00744BF42F0200238
:102ED40022601BB9226822F0200222601022B1E78E
:102EE4007546B3FBF2F002FB1033CB5C05F8013DF1
:102EF40003460028F5D1B7E708681A6810F0800F78
:102F0400496904D0101D18601368196007E010F0B7
:102F1400400F02F1040018601368F6D019800023F2
:102F240075462361B1E71A68111D196015680021FF
:102F34006268284600F0E0F808B1401B60606368EE
:102F44002361002384F843309FE723692A463946E6
:102F54003046C0470130A2D023689B0707D500251F
:102F640004F11909E368039A9B1A9D4205DBE068A2
:102F7400039B9842B8BF184693E701234A46394653
:102F84003046C04701308AD00135EBE7002BA7D18A
:102F94000B7804F1420584F8423065E76232000898
:102FA4005132000838B50023054C05460846236015
:102FB400FEF792FF431C02D1236803B12B6038BD96
:102FC400140A002010B50C46B1F90E1000F0A4F854
:102FD4000028ABBF636DA3891B1823F48053ACBFD7
:102FE4006365A38110BD2DE9F0411F468B89054619
:102FF400DB050C46164605D502230022B1F90E1056
:1030040000F068F8A389324623F48053A381B4F90D
:103014000E103B462846BDE8F04100F017B810B545
:103024000C46B1F90E1000F055F8431CA38915BFE6
:10303400606523F4805343F48053A38118BFA381B4
:1030440010BDB1F90E1000F013B8000038B50546F4
:10305400084611460022054C22601A46FEF764FD1C
:10306400431C02D1236803B12B6038BD140A00202D
:1030740038B50023054C054608462360FEF746FF95
:10308400431C02D1236803B12B6038BD140A00200D
:1030940038B50023064C0546084611462360FEF762
:1030A40038FF431C02D1236803B12B6038BD00BF35
:1030B400140A002038B50023054C05460846236051
:1030C400FEF72CFF431C02D1236803B12B6038BDEB
:1030D400140A002038B50546084611460022054C5E
:1030E40022601A46FEF71CFF431C02D1236803B179
:1030F4002B6038BD140A002010B5C9B202449042B6
:10310400034601D1002010BD1C7801308C42F6D159
:10311400184610BD7047704738B505460846114635
:103124000022054C22601A46FEF7C8FE431C02D159
:10313400236803B12B6038BD140A0020F8B500BF22
:10314400F8BC08BC9E467047F8B500BFF8BC08BC84
:043154009E467047DC
:1031580002030405060708090A0B0C0D0E0F1010D0
:10316800253032782000436865636B2053756D20E5
:103178006572726F72200075706461746520436FA8
:103188006D706C657465200048414C204E4F54208A
:103198004F4B20004572617365204661696C656418
:1031A800200D00626F6F74206C6F6164657220730C
:1031B80074617274006A756D70210000000000006F
:1031C80000000001020304060708090000000001CE
:1031D800020304002000002000000000000000009E
:1031E80000000000000000000000000000000000D7
:1031F80000000000000000000000000000000000C7
:1032080000000000000000000000000000000000B6
:1032180000000000000000000000000000000000A6
:103228000000000000000000000000000000000096
:103238000000000000000000232D302B2000686CE7
:103248004C006566674546470030313233343536C1
:1032580037383941424344454600303132333435FA
:0C32680036373839616263646566000027
:043274000902000843
:04327800E501000864
:10327C000100000010000000BE11030500BEBE0BD3
:10328C00030400EB004000080024F40020000020A0
:10329C00000000000032000820320008E031000875
:1032AC000000000000000000000000000000000012
:1032BC000000000000000000000000000000000002
:1032CC0000000000000000000000000000000000F2
:1032DC0000000000000000000000000000000000E2
:1032EC0000000000000000000000000000000000D2
:04000005080020458A
:00000001FF
